:020000040000FA
:100000008A150A1200280000F20003088301F70095
:100010000A08F8000408F9000B1900000B1800008A
:100020008B180000831203138A110A128C196020A6
:100030000C1B00008C1A00000C1A00000C190000A8
:100040008C1800000C1800000D18000083017908BE
:10005000840078088A0077088300F20E720E090087
:1000C000831603171008110583128A110A120319E7
:1000D0008528AB008A110A122B19CF208A110A1227
:1000E0002B1889208A110A12AB19DB208A110A12F7
:1000F000AB1ABB208A110A12AB18C2208A110A124D
:100100002B1AAF208A110A126028831203138C1154
:100110000800AC01C4018316901190119011901148
:100120000830A100B830A2008830A000C030A6007E
:100130000830A40096019001831203138C118316DA
:100140000317063098003B309100FF3093000130D8
:10015000970083120130AD000313031708008316C4
:1001600011121012101111159514831203138C1112
:1001700003174414080083169012831203138C1182
:1001800003170800831690101208130592018312BA
:1001900003138C110317B000831203170800831692
:1001A00011111011101211169510831203138C11D6
:1001B0000317C40108008317831603171408A03E11
:1001C000840083120008A000840A0008A100840AA9
:1001D0000008A2008316031714089011831203135A
:1001E0008C110317C50020083C39B100243A8A114C
:1001F0000A12031928293108043A8A110A1203192C
:1002000008293108343A8A110A1203198A29080088
:1002100045088A110A12031D1D292E08213A8A1148
:100220000A12031D132983160830A1008830A0008C
:100230008A110A12831282290800083A8A110A12C6
:10024000031D232908004508103A03190800080077
:10025000450818398A110A12031D7B292E08063A0F
:100260008A110A12031D38298A110A127E247A295A
:100270002E08663A8A110A12031D44298A110A12AD
:100280007E248A110A127A292E08053A8A110A1246
:10029000031D50298A110A127B238A110A127A2916
:1002A0002E08033A8A110A12031D59298A110A12CB
:1002B0007A292E08013A8A110A12031D7729270884
:1002C000013A8A110A12031D6B298316191483122D
:1002D0008A110A127A292708023A8A110A12031D82
:1002E0007A2983161A1483128A110A127A298A111A
:1002F0000A126A2D0800083A8A110A12031D812980
:100300000800080083160317A501C830A400831253
:10031000AE0108008317220884000008A300840AA5
:100320000008A400840A0008A500840A0008A600AA
:10033000840A0008A700840A0008A800840A0008AC
:10034000A900840A0008AA0083160830A100A400AE
:1003500083122308213A88300319C8308316A0007D
:1003600015128312AE0123088A110A120319E82913
:100370002308013A8A110A120319032A2308023AB0
:100380008A110A120319182A2308803A8A110A12BC
:100390000319242A2308813A8A110A120319362ADA
:1003A0002308823A8A110A120319482A230860395D
:1003B000203A8A110A120319AD2C23086039403AF9
:1003C0008A110A12031D0C2B8A110A12AC2C080088
:1003D0002408013A8A110A120319872B2408053AC6
:1003E0008A110A1203196F2B2408093A8A110A127A
:1003F00003191C2C2408033A8A110A120319CB2B67
:100400008A110A120C2B2408013A8A110A120319C4
:10041000C82B24080B3A8A110A1203196B2C2408E2
:10042000033A8A110A1203190C2C8A110A120C2B96
:100430002408013A8A110A120319922B2408033A5C
:100440008A110A120319D62B2408083A8A110A12B3
:1004500003190F2C2408063A8A110A120319522A8A
:100460002408003A8A110A120319112B24080A3AA7
:100470008A110A1203194D2C2408003A8A110A1213
:100480000319202B2408063A8A110A120319522A4A
:100490002408003A8A110A1203194B2B8A110A12F6
:1004A0000C2B08002608223A8A110A120319012D82
:1004B0002608213A8A110A1203194F2D02308A00A8
:1004C000031026080339673E03188A0A82000C2BA2
:1004D0006B2A852AB52A0630AE000830B500933065
:1004E000B2000530B3008A110A128D25B400AA08A3
:1004F0008A110A12031D802A29022908031CB4004C
:10050000B40A8A110A127E2408000630AE000310D5
:10051000250D8A110A127925B2000310250D013E1E
:100520007925B3000230B2070318B30A8A110A1200
:100530008D25B4000230B202031CB303AA088A114D
:100540000A120319A62A8A110A12AE2A34082902AD
:100550008A110A120318AE2A2908B4000830B5001F
:10056000B40A8A110A127E2408006630AE002708F9
:100570008A110A12031DC62A2808031DC62A3F3005
:10058000B2000630B3008A110A12FD2A0630B30009
:100590004130B200BB018A110A120326B20A2702B7
:1005A0008A110A12031DDC2A8A110A120326280264
:1005B0008A110A120319E82AB20ABB0A453032022C
:1005C0008A110A12031CCB2AAE018A110A120C2BC3
:1005D000063025028A110A12031CF22AAE018A1182
:1005E0000A120C2B250DB3003B088A110A120926AA
:1005F000B200B30A3B080926B3008A110A12032687
:10060000B40029022908031CB4000830B500B40A5C
:100610008A110A127E240800831603171814831205
:100620000800831626088400831283172D08800093
:10063000840A800183160230A500C830A400080097
:1006400083161708023A8A110A12031D2D2B8312F2
:1006500027088A110A12031D2D2B83161708033A47
:100660008A110A12031D0C2B83122708003C8A11E1
:100670000A12031C0C2B2708383E8400831700083D
:10068000F000831626088400700880000230A50060
:10069000C830A40008000F302705013A8A110A1259
:1006A0000319602B0F302705023A8A110A12031D25
:1006B0000C2B031083161A1803148A110A12642BC8
:1006C0000310831619180314260884008001800D76
:1006D000840A80010230A500C830A4000800250863
:1006E000AF008A110A12AF1B0C2B8A110A12822149
:1006F0000530AE000800AE01AC012F08831696004D
:100700008A110A120319862B023097000800250867
:10071000013A8A110A12031D0C2BAD108A110A121C
:100720008221080025088A110A12031D0C2B2608B5
:10073000031D0C2B831603301705023A8A110A1287
:10074000031DAD2B83120F302705031DAD2B831620
:1007500018108A110A128221080083160330170527
:10076000033A8A110A12031D0C2B83120F3027053E
:10077000023C8A110A12031C0C2B83170F30270529
:100780008316983E840000108A110A128221080004
:100790008A110A120C2B2508013A8A110A12031D2C
:1007A0000C2BAD148A110A128221080025088A1127
:1007B0000A12031D0C2B2608031D0C2B8316033075
:1007C0001705023A8A110A12031DF12B83120F300A
:1007D0002705031DF12B831618148A110A12822192
:1007E0000800831603301705033A8A110A12031D05
:1007F0000C2B83120F302705023C8A110A12031CAE
:100800000C2B83170F3027058316983E84000014A5
:100810008A110A12822108008A110A120C2B8316EF
:1008200026088400831283172C0880008316013069
:10083000A500C830A40008002508013C8A110A124E
:10084000031C0C2B2508AC008A110A1203192B2C4F
:100850008316033097008A110A1282218316031728
:10086000C830AA000830A9008830A8000830AD00C0
:10087000D030AE004830AC00D830B2000830B10003
:100880008830B0000830B500D830B6004830B40029
:100890000E3099000E309A00080083161708033AAC
:1008A0008A110A12031D0C2B83122708003C8A119F
:1008B0000A12031C0C2B2708383E840083170008FB
:1008C000F000831626088400700880000130A5001F
:1008D000C830A40008008316170883120339033AAE
:1008E0008A110A12031D0C2B2708383E8400831737
:1008F000250880008A110A12822108008316031736
:1009000083172608840083120317B70137083502BE
:100910008A110A120319A02C8A110A12B40B932C03
:100920008A110A129F2C8A110A128D258000B70A9B
:10093000840A8A110A12B20F862CB30A862CAE01E1
:1009400037088316A5004030240640398838A400B3
:0A0950008A110A12080008000800CE
:06095A008A110A122308B5
:10096000213A0319D42C8A110A122308223A0319B6
:10097000712D8A110A122308233A0319712D8A1145
:100980000A122308A13A0319712D8A110A122308A9
:10099000A23A0319712D8A110A122308A33A0319E6
:1009A000712D8A110A120C2B2408013A8A110A129D
:1009B0000319712D2408023A8A110A120319712DA4
:1009C0002408033A8A110A120319712D2408063AE1
:1009D0008A110A120319012D2408093A8A110A12F0
:1009E0000319742D24080A3A8A110A120319712D69
:1009F00024080B3A8A110A120319712D8A110A125E
:100A00000C2B831203170630AE000830B500260801
:100A1000013A8A110A120319202D0310270D8A1199
:100A20000A128325B2000310270D013E8325B3006F
:100A30008A110A128D25B400B20A8A110A12402DB9
:100A40002608023A8A110A120319392D0310270DBC
:100A50008A110A128325B2000310270D013E832557
:100A6000B3008A110A128D25B400B20A8A110A1243
:100A7000402D2608033A8A110A1203190C2B08008C
:100A80002A088A110A12031D4A2D2908340229084E
:100A90000318B400B40A8A110A127E240800063032
:100AA000AE000830B500B730B2000530B3008A118F
:100AB0000A128D25B400AA088A110A12031D642D9A
:100AC00029022908031CB400B40A8A110A127E24E0
:100AD000080008008A110A122E08063A03197E241B
:100AE00008008A110A120C2B2130AE00831603175E
:100AF0000800F00005308A008130700703188A0A68
:100B00008200A5340534F00005308A008B30700770
:100B100003188A0A8200CE3405348312031733087F
:100B20008A00320882001234013400340134003467
:100B3000003400340834003400340134003400340C
:100B400000340234013400340134093402342934CD
:100B50000034013401340434803432340934043430
:100B600000340034023403340034003400340934D7
:100B7000213400340134003401342234343400345C
:100B80000734053481340334083400340A3407341C
:100B9000053401340334083400340A343434063460
:100BA000A034FF3409340134A1340134093402344F
:100BB000A13400340634A134FF3409340334093439
:100BC00004341534803425347F34353400344534CE
:100BD000FF347534083495340834813402340934D0
:100BE0000534093406341534803425347F343534E3
:100BF00000344534FF347534083495340834913466
:100C00000234C034C0348312031733088A00320818
:100C10008200F0000310F00D8A110A121C26B600A3
:100C2000F00A8A110A121C26F00070088A003608A1
:100C3000330703188A0A820006308A0023307007BF
:100C400003188A0A820027340634333406343F34CA
:100C5000063445340634613406347D340634893430
:100C60000634933406343F340634A3340634B734A0
:100C70000634E5340634F1340634FB3406340634E5
:100C8000033409340434043408341C340334493440
:100C900000344F340034433400346134003472344F
:100CA0000034643400345334003474340034653414
:100CB00000347034003470340034653400347234DD
:100CC00000341C3403344D340034613400346E3449
:100CD000003475340034653400346C34003420340E
:100CE000003456340034653400346C3400346534D8
:100CF00000347A340034203400340C340334563455
:100D00000034313400342E34003430340034303484
:100D100000340A3403344334003466340034673416
:100D2000003431340034103403344E3400346F3422
:100D300000347434003468340034693400346E3460
:100D4000003467340034143403344D3400346934CF
:100D5000003463340034723400346F34003463344C
:100D600000346834003469340034703400342E3474
:100D70000334503400346934003463340034313483
:100D800000343634003443340034373400343634DD
:100D900000343534003420340034553400345334B6
:100DA00000344234003420340034493400344F34A9
:100DB0000034433400346134003472340034643419
:100DC000003473340034203400340C34033456348B
:100DD0000034313400342E340034303400343034B4
:100DE00000340A3403344334003466340034673446
:100DF000003431340034103403344E3400346F3452
:100E000000347434003468340034693400346E348F
:060E1000003467340034D9
:101000001E30F200F20B02288316031381178A1593
:101010000A128025831603178A150A12640003300A
:101020001705033A031D0E28831203138501860159
:10103000FB018701FC01F6018A150A12E1228A15DB
:101040000A12831320308400083046248A150A12BD
:10105000031C31288A150A123A22831203136E30B8
:10106000FA0283120313F6088A150A120319B0282C
:10107000831203138A150A12A808031D9D28013044
:1010800083120313FD080319FE00831203138A154C
:101090000A12A908031D6928831203137E08F400AD
:1010A000F403831603130C13831203139F171F13E8
:1010B0009F121F129F1174189F15F4181F16F41811
:1010C0009F151F14831203130130A9008A150A12F9
:1010D0009B288A150A12291C7728831203131F15CF
:1010E000831203130230A9008A150A129B288A155D
:1010F0000A12A91C9B28831203138A150A121F19AE
:101100009B2883120313A901831203130C13831268
:101110000313FD0803199B28831203131E0883126F
:101120000313A1007E08A000FE038A150A12031D06
:101130009B287D08FE002D30A8008A150A12CC20BD
:101140008A150A1246218A150A12C0218A150A1226
:10115000352483120313FF30FA0083120313A8030C
:10116000831203138A150A12A00803191F288A156F
:101170000A12831383120313203084000830CA2418
:101180008A150A12031CB728831203135A30FA0275
:10119000A0018A150A121F28AB088A150A12031922
:1011A000D728AE038A150A1203192B290800320822
:1011B000AB00AB088A150A120319EA28B201AD0187
:1011C0008A150A12AB1FD1282D143202AB008A15E2
:1011D0000A12D1288A150A12AF080319D6288312D9
:1011E0000313050883120313F4008A150A122F1C37
:1011F000FF288A150A12741D2129AF01AF148A1520
:101200000A12AF1C09298A150A1274192129AF0183
:101210002F158A150A122F1D13298A150A12741DFB
:101220002429AF01AF158A150A1274192429AF01B8
:101230003008A2003108A300FF30A0080319A00065
:1012400008000130AB0008000130AB000310B0070C
:101250000318B10A0800831203132C08AE00AE0A6B
:1012600083120313340884008A150A122D184029AA
:101270008A150A1296230408B4008A150A12D62881
:101280008A150A12AE238A150A123B29C2088A154A
:101290000A1203195129C5038A150A120319A5292F
:1012A00008004908C200C2088A150A1203196429F5
:1012B000C901C4018A150A12C21F4B2944144902EC
:1012C000C2008A150A124B298A150A12C608031988
:1012D000502983120313050883120313F4008A159F
:1012E0000A12461C79298A150A12741E9B29C60106
:1012F000C6148A150A12C61C83298A150A12741A82
:101300009B29C60146158A150A12461D8D298A1584
:101310000A12741E9E29C601C6158A150A12741A6D
:101320009E29C6014708A4004808A500FF30A00870
:101330000319A00008000130C20008000130C200FB
:101340000310C7070318C80A0800831203134308D1
:10135000C500C50A831203134B0884008A150A12BC
:101360004418BA298A150A12CB230408CB008A151F
:101370000A1250298A150A12E3238A150A12B5297E
:10138000D9088A150A120319CB29DC038A150A1217
:1013900003191F2A08006008D900D9088A150A1203
:1013A0000319DE29E001DB018A150A12D91FC529BC
:1013B0005B146002D9008A150A12C5298A150A121F
:1013C000DD080319CA2983120313050883120313C6
:1013D000F4008A150A125D1CF3298A150A12F41EFC
:1013E000152ADD01DD148A150A12DD1CFD298A1576
:1013F0000A12F41A152ADD015D158A150A125D1DFF
:10140000072A8A150A12F41E182ADD01DD158A152D
:101410000A12F41A182ADD015E08A6005F08A70068
:10142000FF30A0080319A00008000130D90008000F
:101430000130D9000310DE070318DF0A0800831209
:1014400003135A08DC00DC0A8312031362088400C9
:101450008A150A125B18342A8A150A120024040815
:10146000E2008A150A12CA298A150A1218248A1556
:101470000A122F2A831203130130F6008A150A126A
:10148000A61B452A2608FD00FE008A150A12A01B8D
:10149000602A8A150A12A1080319762A2008AC00CE
:1014A000AC132C13031021088A150A12201B5C2A86
:1014B000B2078A150A12762AB2028A150A12762A09
:1014C0008A150A12201B702A2008AC00AC132C13BA
:1014D0000130AF00AD00B001B1018A150A12762AC1
:1014E000083083120313B3003930B4008A150A128E
:1014F000A21B912A8A150A12A3080319A72A2208F7
:10150000C300C3134313031023088A150A12221BB6
:101510008D2AC9078A150A12A72AC9028A150A1232
:10152000A72A8A150A12221BA12A2208C300C31364
:1015300043130130C600C400C701C8018A150A124E
:10154000A72A083083120313CA005030CB008A1533
:101550000A12A41BC22A8A150A12A5080319D82A3E
:101560002408DA00DA135A13031025088A150A1220
:10157000241BBE2AE0078A150A12D82AE0028A151F
:101580000A12D82A8A150A12241BD22A2408DA0041
:10159000DA135A130130DD00DB00DE01DF018A15AA
:1015A0000A12D82A083083120313E1006730E200E0
:1015B000A001A101A201A301A401A501A601A70107
:1015C000080083160313FF3085000030860080304A
:1015D00087008316031304309F00831203139F17A1
:1015E0001F13831603130C13831203138601FB01CD
:1015F000870183120313FD01FE01A801A901A001C7
:10160000FF30FA00831203130130B5000230B60038
:101610000430B7000830B800831203130130B9005A
:101620000330BA000230BB000630BC000430BD00FD
:101630000C30BE000830BF000930C0008312031315
:101640001030CC002030CD004030CE008030CF00B4
:10165000831203131030D0003030D1002030D2007C
:101660006030D3004030D400C030D5008030D60088
:101670009030D700831203130130E3000230E400FE
:101680000430E5004030E600831203130130E70028
:101690000330E8000230E9000630EA000430EB00D5
:1016A0004430EC004030ED004130EE00AB01AD01C4
:1016B000AF01B201AC01AE01AE0A0430B30001309B
:1016C000AA003530B400C201C401C601C901C3017A
:1016D000C501C50A0430CA000130C1004C30CB003E
:1016E000D901DB01DD01E001DA01DC01DC0A0430B3
:1016F000E1000130D8006330E200080083120313D8
:10170000FD08031908007E08F400F4038316031390
:101710000C13831203139F121F129F1174189F152D
:10172000F4181F16F4189F151F14080083120313D2
:10173000AB03840AAA0A2A08031033028A150A1284
:10174000031CA52B8A150A12C32B0130AA003530C1
:10175000331D393084008A150A12C32B83120313F8
:10176000AB038403AA038A150A120319BA2B8A153C
:101770000A12C32B3308AA003830331D40308400CE
:101780008A150A12C32B831203137B08F039000455
:10179000FB008600080083120313C203840AC10AF7
:1017A000410803104A028A150A12031CDA2B8A1513
:1017B0000A12F82B0130C1004C304A1D5030840011
:1017C0008A150A12F82B83120313C2038403C10380
:1017D0008A150A120319EF2B8A150A12F82B4A08E8
:1017E000C1004F304A1D573084008A150A12F82B69
:1017F000831203137B080F390004FB0086000800E6
:1018000083120313D903840AD80A5808031061020B
:101810008A150A12031C0F2C8A150A122D2C01306E
:10182000D8006330611D673084008A150A122D2CA0
:1018300083120313D9038403D8038A150A120319E8
:10184000242C8A150A122D2C6108D8006630611DDF
:101850006E3084008A150A122D2C831203137C0823
:1018600000390004FC00870008000130F4008312F6
:1018700003137A08F500000000008A150A12F50B20
:0C1880003B2C8A150A12F40B372C0800D0
:04188C0003088312B8
:101890000317C3000408BD00831603178A150A1234
:1018A000A81B822C290883120317C100C2008A15C5
:1018B0000A120319722C831603172A0883120317BE
:1018C000BE0083173E0884000008F1003D08840034
:1018D000C31F831371088000BD0ABE0A8A150A124D
:1018E000C10B612C831628084039403A8838A8007B
:1018F0000830A90083124208F100430883007108F0
:101900000314080083120317430883000310080020
:10191000030883120317C3000408BD0083160317CE
:101920008A150A12B01BC42C310883120317C10098
:10193000C2008A150A120319B42C83160317320841
:1019400083120317BE0083173E0884000008F100CD
:101950003D088400C31F831371088000BD0ABE0ABE
:101960008A150A12C10BA32C831630084039403A5D
:101970008838B0000830B10083124208F1004308F3
:1019800083007108031408008312031743088300BF
:1019900003100800F100030883120317C300710845
:1019A0000F39C1000408BE004108831603178A15C9
:1019B0000A12AC1B012DAD008A150A120319F52C71
:1019C0002E088312BD008317C31F83133E088400B3
:1019D0000008F10083173D08840071088000BD0AEB
:1019E000BE0A8A150A12C10BE32C83162C08403953
:1019F000403A8838AC00831203174308830003146D
:101A0000080003100800F100030883120317C30045
:101A100071080F39C1000408BE004108831603177E
:101A20008A150A12B41B3A2DB5008A150A12031939
:101A30002E2D36088312BD008317C31F83133E0863
:101A400084000008F10083173D08840071088000BD
:101A5000BD0ABE0A8A150A12C10B1C2D8316340852
:101A60004039403A8838B400831203174308830092
:101A7000031408000310080083170339983E8400FC
:101A80000014080083170339983E840000100800F2
:101A900083120317441C08008316101111159514A6
:101AA000630000009510101211161011111108009A
:101AB00083120317AD1C080083169510111610121F
:101AC0001111101115158312BB018030BC008A154D
:101AD0000A12BB0B692DBC0B692D8316151108006A
:101AE0008316031795118312BC01BB018A150A12D4
:101AF000BB0F782DBC0F782D8A150A12802508009F
:101B0000831603179701013091009001083095006A
:101B10008312AC010130AD00B801B901BA01FF3048
:101B2000AE00831203138C1183168C150B178B17C1
:101B300008008316031795119514970103138C1150
:021B400008009B
:044000000034003454
:02400E00FA3F77
:00000001FF
